:100000000C9454080C9474080C9474080C947408A0
:100010000C9474080C9474080C9474080C94740870
:100020000C9474080C9474080C9474080C94740860
:100030000C9474080C9474080C9474080C94740850
:100040000C9474080C9463130C9474080C94740846
:100050000C9474080C9474080C9474080C94740830
:100060000C9474080C94012C0C94CD2B0C947408F3
:100070000C9474080C9485080C9474080C947408FF
:100080000C9474080C9474080C9474080C94740800
:100090000C9474080C9474080C9474080C947408F0
:1000A0000C9474080C9474080C9474080C947408E0
:1000B0000C9474080C9474080C9474080C947408D0
:1000C0000C9474080C9474080C9474080A737720C8
:1000D000310A000A737720300A00414D433A206EFE
:1000E0006F77204D300A00414D433A206E6F7720E4
:1000F0004D310A00414D433A2068616E646C6520C1
:10010000636C6F7365640A00414D433A204D3120A2
:1001100068616E646C652073746174757320636FBD
:100120007272656374696F6E0A00414D433A206EC6
:100130006F77204D320A00414D433A2068616E646A
:100140006C65206F70656E65640A00414D433A200E
:100150006E6F77204D330A00414D433A2068616E3F
:10016000646C65206F70656E65640A00414D433AAA
:10017000206E6F77204D340A00414D433A2068616C
:100180006E646C65206F70656E65640A00414D4356
:100190003A204D342068616E646C6520737461741C
:1001A000757320636F7272656374696F6E0A0041C4
:1001B0004D433A206E6F77204D350A00414D433A4A
:1001C0002068616E646C6520636C6F7365640A00FF
:1001D000414D433A206E6F77204D360A000A414D5B
:1001E00043206873776170206F75743A20000A535A
:1001F0004953383330304C0A004275696C742077AB
:10020000697468204156522D4743433A2000342EEA
:10021000362E320020616E64204156522D4C4942E8
:10022000433A2000312E382E30002072656C656113
:1002300073653A20003230313131323238000A6F82
:100240006E20004175672032342032303136002074
:100250002F200031313A32353A3532000A0A004156
:100260004D43207374617475733A204D000A005237
:10027000544D207374617475733A204D000A0A005E
:1002800020436F6D6D616E646C6973743A0A20531C
:10029000544154202D204669726D77617265205259
:1002A00065766973696F6E2C205374617475732C55
:1002B000206574632E2E2E0A2048454C50202D2098
:1002C0007468697320706167650A002072746D201C
:1002D0007A6F6E65333A200020616D63207A6F6E0D
:1002E00065333A20002072746D206D617463683A42
:1002F00020002072746D20636C6F7365640A0020A7
:1003000072746D206F70656E65640A002072746D82
:10031000206F70656E65640A002072746D206F70C6
:10032000656E65640A002072746D206F70656E657D
:10033000643A2000505752202B3132563A20002088
:100340006D560A4420202B332E33563A20200020AD
:100350006D560A4420202B322E35563A202000209C
:100360006D560A4420202B312E35563A202000208D
:100370004572617375726520454550524F4D202E70
:100380002E2E200020577269746520414435333386
:10039000383A2000205265616420414435333338B7
:1003A0000069326320627573206572726F720A0091
:1003B000756E6B6E6F776E20693263207374617433
:1003C000652000657272207374613A200065727254
:1003D00020736C613A2000657272206474613A2067
:1003E000000A0A534953383330304C206465627533
:1003F000672070726F6D70740A000A00574454438E
:1004000053523A20000A004D4D432046573A2000EF
:100410000A4275696C742077697468204156522DC0
:100420004743433A2000342E362E320020616E645A
:10043000204156522D4C4942433A2000312E382E4D
:1004400030002072656C656173653A20003230318E
:100450003131323238000A6F6E2000417567203228
:1004600034203230313600202F200031313A3235FD
:100470003A3533000A004D435553523A20000A00E2
:100480007265737461727420616674657220636F43
:100490006C642072657365740A004D4F4453544177
:1004A00054455F504F5745524544202D3E204D4FF7
:1004B0004453544154455F574149545F5245534555
:1004C0005420000D0A004D4F4453544154455F578A
:1004D0004149545F5245534554202D3E204D4F44D1
:1004E00053544154455F574149545F465047415F1B
:1004F000444F4E4520000D0A004D4F445354415483
:10050000455F574149545F465047415F444F4E4510
:10051000202D3E204D4F4453544154455F46504793
:10052000415F52445920000D0A004D4F445354413D
:1005300054455F465047415F52445920000D0A0020
:10054000708A728E9290748C76989C9AA0A4889EE1
:10055000868478947A9682807C7EA207005101314D
:10056000000006C10003540201FF7F00703F00003D
:10057000040000620200040CC0077FEFABFF00C163
:10058000B7AD8A8F940202000000C6442B312E358D
:10059000560000000000000000000006005101317C
:1005A000000005C10003540201FF7F00703F0000FE
:1005B0000400007A0200040CC0077FEFABFF00F7D5
:1005C000F2E9A2A7AB0202000000C6442B322E358E
:1005D0005600000000000000000000020051013041
:1005E000000001C10003540101FF7F00703F008043
:1005F000010000010600040C00001946007DC955E9
:10060000504600050A0505000000C57446504741E4
:100610000000000000000000000000000051111662
:100620000001002B000000C00000CB5349533833B9
:1006300030304C52544D00005112130000002B007A
:100640000000C10000C8534953383330304C020019
:1006500051012F000008C00003540101FF7F00700A
:100660003F0080010000010600040C000019460054
:100670007DC955463C00050A0505000000C47452BA
:10068000544D0000000000000000000000000100C8
:10069000510135000007C0000340F26F0700000061
:1006A0000700000000000000000000000000000043
:1006B00000000000000000000000000000CA486FB9
:1006C000745377617052544D000000000000050023
:1006D000510131000004C10003540201FF7F00708A
:1006E0003F0000040000A10200040CC0077FEFAB34
:1006F000FF00F7F2E9A2A7AB0202000000C6442BFC
:10070000332E3356000000000000000000000400FB
:10071000510132000003C10003540201FF7F007049
:100720003F0000040000360200040CD0077FEFAB4E
:10073000FF00F7F2E9A2A7AB0202000000C7505782
:10074000522B313256000000000000000000030070
:10075000510131000002C10003540101FF7FFF7FFE
:100760003F0080010000010600040C0000193C322B
:1007700078E755463C00050A0505000000C67450A0
:100780006F776572000000000000000000000100AB
:10079000510132000000C1000340F26F0700000069
:1007A0000700000000000000000000000000000042
:1007B00000000000000000000000000000C7486FBB
:1007C0007453776170000000000000000000707238
:1007D0006F633A204E4554464E5F4150503A204395
:1007E0004D445F4745545F4445564943455F49443E
:1007F0000A0070726F633A204E4554464E5F53456F
:100800004E535F4556454E543A20434D445F534541
:10081000545F4556454E545F5245434549564552EF
:100820000A0070726F633A204E4554464E5F53453E
:100830004E535F4556454E543A20434D445F47451D
:10084000545F4556454E545F5245434549564552BF
:100850000A0070726F633A204E4554464E5F53450E
:100860004E535F4556454E543A20434D445F504CDD
:100870004154464F524D5F4556454E540A007072E2
:100880006F633A204E4554464E5F53454E535F4585
:1008900056454E543A20434D445F4745545F4445C6
:1008A000564943455F5344525F494E464F0A0070D4
:1008B000726F633A204E4554464E5F53454E535F28
:1008C0004556454E543A20434D445F4745545F4496
:1008D00045564943455F5344520A0070726F633A6C
:1008E000204E4554464E5F53454E535F4556454E48
:1008F000543A20434D445F5245535F444556494363
:10090000455F5344525F5245500A0070726F633A1C
:10091000204E4554464E5F53454E535F4556454E17
:10092000543A20434D445F4745545F53454E534F1F
:10093000525F52454144494E470A0070726F633A14
:10094000204E4554464E5F53454E535F4556454EE7
:10095000543A20434D445F4745545F53454E534FEF
:10096000525F5448524553484F4C44530A007072EA
:100970006F633A204E4554464E5F53454E535F4594
:1009800056454E543A20756E6B6E6F776E3A200066
:1009900070726F633A204E4554464E5F53544F5227
:1009A0004147453A20434D445F4745545F465255C1
:1009B0005F494E565F415245415F494E464F0A00DE
:1009C00070726F633A204E4554464E5F53544F52F7
:1009D0004147453A20434D445F524541445F4652AA
:1009E000555F444154413A2000414D430A0052545E
:1009F0004D0A0070726F633A204E4554464E5F5365
:100A0000544F524147453A20434D445F5752495451
:100A1000455F4652555F444154413A2000414D43A1
:100A20000A0052544D200070726F633A204E4554B4
:100A3000464E5F5049434D473A20434D445F47453A
:100A4000545F5049434D475F50524F50530A007016
:100A5000726F633A204E4554464E5F5049434D47AE
:100A60003A20434D445F4652555F434F4E54524FD8
:100A70004C3A2000414D430A0052544D0A00707216
:100A80006F633A204E4554464E5F5049434D473AB6
:100A900020434D445F4745545F4652555F4C4544A3
:100AA0005F50524F50530A0070726F633A204E45A8
:100AB00054464E5F5049434D473A20434D445F47AB
:100AC00045545F4C45445F434F4C4F525F43415048
:100AD00041420A0070726F633A204E4554464E5FA1
:100AE0005049434D473A20434D445F5345545F4678
:100AF00052555F4C45445F53544154450A0070724F
:100B00006F633A204E4554464E5F5049434D473A35
:100B100020434D445F4745545F4652555F4C454422
:100B20005F53544154450A0070726F633A204E453A
:100B300054464E5F5049434D473A20434D445F472A
:100B400045545F4652555F4C45445F5354415445AC
:100B5000206572723A000A0070726F633A204E4547
:100B600054464E5F5049434D473A20434D445F47FA
:100B700045545F4445565F4C4F4341545F52454393
:100B80005F49440A0070726F633A204E4554464EE6
:100B90005F5049434D473A20434D445F4652555FAD
:100BA000434F4E54524F4C5F43415041420A0070F4
:100BB000726F633A204E4554464E5F5049434D474D
:100BC0003A20434D445F5345545F414D435F504F7E
:100BD00052545F53544154450A0070726F633A2077
:100BE0004E4554464E5F5049434D473A20434D448D
:100BF0005F4745545F414D435F504F52545F5354DC
:100C00004154450A0070726F633A204E4554464E77
:100C10005F5049434D473A20434D445F4745545F39
:100C2000434C4F434B5F53544154450A0070726F1D
:100C3000633A204E4554464E5F5049434D473A2053
:100C4000434D445F5345545F4652555F41435449B9
:100C5000564154494F4E0A0070726F633A204E4518
:100C600054464E5F5049434D473A20434D445F53ED
:100C700045545F504F5745525F4C4556454C0A000E
:100C800070726F633A204E4554464E5F5049434D53
:100C9000473A20756E6B6E6F776E0A0070726F63E5
:100CA0003A204E4554464E5F56454E444F523A20E8
:100CB000434D445F524541445F52544D5F45450AA0
:100CC0000070726F633A204E4554464E5F56454E53
:100CD000444F523A20434D445F57524954455F5266
:100CE000544D5F45450A0070726F633A204E45547B
:100CF000464E5F56454E444F523A20434D445F4D59
:100D00004F444946595F52544D5F45455F57500A1D
:100D10000070726F633A204E4554464E5F56454E02
:100D2000444F523A20434D445F52455345545F4629
:100D30005047410A0070726F633A204E4554464E48
:100D40005F56454E444F523A20434D445F47455409
:100D50005F4649524D575F56455253494F4E0A0020
:100D600070726F633A204E4554464E5F56454E446E
:100D70004F523A20434D445F4745545F75445743B3
:100D80005F4441435F56414C55450A0070726F63A2
:100D90003A204E4554464E5F56454E444F523A20F7
:100DA000434D445F5345545F754457435F4441434B
:100DB0005F56414C55450A0070726F633A204E45AC
:100DC00054464E5F56454E444F523A20434D445F81
:100DD000524541445F52544D5F54454D505F56411A
:100DE0004C55450A0070726F633A204E4554464E8A
:100DF0005F56454E444F523A20434D445F5345544D
:100E00005F52544D5F54454D505F504F494E0A005C
:100E100070726F633A204E4554464E5F56454E44BD
:100E20004F523A20464F4F200A0052544D3A206EFE
:100E30006F77204D300A0052544D204D61736B3A4C
:100E4000200052544D3A204552524F523A204932D6
:100E500043206275732053444120737475636B2083
:100E60006C6F770A0052544D3A20636F6D70617455
:100E70006962696C69747920636865636B3A200004
:100E80006D730A0052544D3A206E6F77204D310A2F
:100E900000636F6D702E20636865636B3A20737515
:100EA00063636573730A00636F6D702E20636865FA
:100EB000636B3A206E6F206D6174636865732066A2
:100EC0006F756E640A0052544D204D61736B3A2069
:100ED000000A0052544D3A2068616E646C652063CC
:100EE0006C6F7365642C20656467650A0052544D0D
:100EF0003A2068616E646C6520636C6F7365642C66
:100F0000204D30206C6576656C0A0052544D3A20B5
:100F10006D6F64756C652072656D6F7665640A002F
:100F200052544D3A206E6F77204D320A0052544D84
:100F3000204D61736B3A200052544D3A2068616E27
:100F4000646C65206F70656E65640A0052544D3A9A
:100F5000206D6F64756C652072656D6F7665640ACF
:100F60000052544D3A206E6F77204D330A00525490
:100F70004D3A206E6F77204D340A0052544D204D6B
:100F800061736B3A200052544D3A2053657475706A
:100F9000204457435F44414320746F203256350A42
:100FA0000052544D3A2068616E646C65206F706524
:100FB0006E65640A0052544D3A206D6F64756C651D
:100FC0002072656D6F7665640A0052544D3A205365
:100FD0006574646F776E204457435F4441430A0051
:100FE00052544D3A206E6F77204D350A0052544DC1
:100FF000204D61736B3A200052544D3A2053657472
:10100000646F776E204457435F4441430A00525453
:101010004D3A206D6F64756C652072656D6F7665F5
:10102000640A0052544D3A206E6F77204D360A0004
:1010300052544D204D61736B3A200052544D3A206A
:101040006D6F64756C652072656D6F7665640A00FE
:101050000A616D6320776974686F7574207A332034
:101060007265636F7264730A000A72746D20776927
:1010700074686F7574207A33207265636F7264735D
:101080000A000A666F7220616D633A2000666F7213
:101090002072746D3A20000A52544D2068737761B3
:1010A00070206F75743A200011241FBECFEFD1E27B
:1010B000DEBFCDBF13E0A0E0B2E0E4EFFFE500E06B
:1010C0000BBF02C007900D92AA3FB107D9F71BBE14
:1010D0001AE0AAEFB3E001C01D92A938B107E1F709
:1010E0000E94E92C0C94F82F0C9400001092390403
:1010F00010927C0087EC80937A0080917A0084FFC4
:10110000FCCF8FEC80937A0008951F920F920FB658
:101110000F920BB60F9211242F934F935F936F93FF
:101120007F938F939F93AF93BF93EF93FF938091A0
:10113000780090917900A0E0B0E04091FA035091DE
:10114000FB036091FC037091FD03840F951FA61FA4
:10115000B71F8093FA039093FB03A093FC03B09313
:10116000FD032091FE032F5F2093FE032223E9F469
:1011700020913904E22FF0E0EE0FFF1FEF5CFB4FF0
:10118000892F9A2FAB2FBB27918380831092FA036C
:101190001092FB031092FC031092FD03822F8F5FCD
:1011A00083708093390480937C008FEC80937A0065
:1011B000FF91EF91BF91AF919F918F917F916F912F
:1011C0005F914F912F910F900BBE0F900FBE0F901C
:1011D0001F901895E82FF0E0E370F070EE0FFF1FFE
:1011E000EF5CFB4F8081918108951F93CF93DF9334
:1011F000CDB7DEB7C354D0400FB6F894DEBF0FBEF4
:10120000CDBF182F8DED91E00E943B2C812F0E94C5
:10121000B42C80E092E00E94292C809162098C839A
:1012200080E18D83809117098F8380916109888780
:101230008C5F8093610982E0898784E08A8782EFEE
:101240008B871C868FE68D871E878BE08B83CE0174
:1012500001960E941B1481E08A83CE0101960E94B0
:10126000DD1010930202CD5BDF4F0FB6F894DEBFA6
:101270000FBECDBFDF91CF911F910895CF9380E82E
:101280000E943A2BC82F8091040280930302809120
:1012900005048093040280910604C81749F0CC230A
:1012A00019F08CEC90E002C083ED90E00E943B2CA2
:1012B00080E80E943A2B90910404882319F09D7FC6
:1012C000916002C092609E7F90930404809104021A
:1012D000833009F482C0843040F49091030281305D
:1012E00071F1823008F058C00AC0853009F4D3C0CB
:1012F000853008F498C0863009F00DC1F0C09923FC
:1013000009F406C18AED90E00E943B2C80E060E089
:1013100041E050E00E941B1181E060E041E050E0BC
:101320000E941B1182E060E043E050E00E941B112C
:1013300082E060E040E050E00E941B11E9C0913083
:1013400051F080E060E041E050E00E941B1187EE28
:1013500090E00E943B2C80910604C81771F0CC23CA
:1013600061F0C093060484EF90E00E943B2C80E083
:101370000E94F50882E08093050480910604C81756
:1013800009F445C0CC2309F042C01092060488E05D
:1013900091E00E943B2C3BC0923021F08AE291E028
:1013A0000E943B2C80910604C81771F0CC2361F495
:1013B0001092060487E391E00E943B2C81E00E949A
:1013C000F50881E08093050480910304882309F4E3
:1013D000A2C01092030483E09CC08091030283307A
:1013E00021F08BE491E00E943B2C80910604C81709
:1013F00071F0CC2361F41092060488E591E00E941C
:101400003B2C81E00E94F50881E0809305048091E7
:101410000204882309F47FC01092020481E08093C3
:10142000160984E076C080910302843021F08CE6B6
:1014300091E00E943B2C80910604C81781F0CC23D8
:1014400071F41092060489E791E00E943B2C81E040
:101450000E94F50885E08093050410920E098091A2
:101460000604C81741F0CC2331F0C09306048DE880
:1014700091E00E943B2C80910004882309F44BC02A
:101480001092000487E08093160986E0809305049B
:1014900010920E0940C080910302853021F08FEA3E
:1014A00091E00E943B2C80910604C81771F0CC2378
:1014B00061F0C09306048CEB91E00E943B2C80E02D
:1014C0000E94F50884E0809305048091010488233C
:1014D00079F01092010486E08093050409C08091A0
:1014E0000302863029F00D9A80ED91E00E943B2C9A
:1014F00080910004882329F01092000487E08093F3
:10150000160980911609882331F482E00E94F508BB
:1015100081E0809305048091FF03882329F1809165
:10152000040480FF03C080E00E94F5088091040459
:1015300081FF03C081E00E94F5088091040482FFCE
:1015400003C082E00E94F5088091040483FF03C079
:1015500083E00E94F5088091040484FF03C084E0C6
:101560000E94F5081092FF03CF9108958091040224
:10157000089580910404089581E080930304089500
:1015800081E08093020410920104109200040895F7
:1015900081E08093010410920204109200040895E7
:1015A00081E08093000410920104109202040895D7
:1015B00081E08093FF0308956F927F928F929F92B4
:1015C000AF92BF92CF92DF92EF92FF920F931F9351
:1015D000CF93DF93CDB7DEB7C850D1400FB6F894A4
:1015E000DEBF0FBECDBF4C01E62E3A01FC011082DA
:1015F000CE01019660E070E048E050E00E94C82F04
:10160000FE01319697E080E02191820F9150E1F741
:1016100081959885891709F059C00E8110E093E0F3
:10162000000F111F9A95E1F70115110509F450C03B
:1016300089E0A82EB12CAC0EBD1EB80160507040E0
:10164000CE01019645E050E00E94C82F8A81998121
:10165000890FFB808F0D9C81890F81959D81891752
:10166000C9F5CF2CDD240B5F1F4FB80160507040CF
:10167000C501A6010E94C82F20E030E006C08A0DF7
:101680009B1DFC018081280F3F5F832F90E08C150C
:101690009D05A8F321958C812817F1F48C85803362
:1016A00079F4F40180818F5F80838E1549F4611491
:1016B000710431F0C301B5014F2D50E00E94BF2FDE
:1016C0008A8187FD0BC00C0D1D1DB7CF82E007C0BE
:1016D00083E005C084E003C085E001C080E0C85F0E
:1016E000DE4F0FB6F894DEBF0FBECDBFDF91CF91B6
:1016F0001F910F91FF90EF90DF90CF90BF90AF9030
:101700009F908F907F906F900895EF92FF920F932C
:101710001F93CF93DF93CDB7DEB728970FB6F8941A
:10172000DEBF0FBECDBF7C01CE01019660E070E050
:1017300048E050E00E94C82FFE01319697E080E01B
:101740002191820F9150E1F781959885891749F58C
:101750000E8110E023E0000F111F2A95E1F701151B
:10176000110509F1B80160507040CE01019645E0C5
:1017700050E00E94C82F2A819981920F8B81980F87
:101780003C81930F91953D81931779F490E00596F4
:10179000080F191F27FFE6CFF7011183008380E0B0
:1017A00005C082E003C083E001C084E028960FB644
:1017B000F894DEBF0FBECDBFDF91CF911F910F9187
:1017C000FF90EF90089589E193E00E943B2C80E028
:1017D000089580E892E00E943B2C80E00895CF932A
:1017E000DF9300D0CDB7DEB784E993E00E943B2CB5
:1017F0008CE061E0AE014F5F5F4F0E941C2988239F
:1018000029F085E092E00E94292C0AC08DE092E048
:101810000E94292C89810E94B42C8A810E94B42CB8
:1018200082E192E00E94292C80E00F900F90DF91DE
:10183000CF910895CF93DF9300D000D0CDB7DEB71E
:1018400019821A821B821C828CE289838CE18A8332
:10185000A0E7B4E0FE01319680E090E03D91232FB7
:1018600020532A3008F027502193019684309105A7
:10187000A9F789818295807F9A819F70892B8983BE
:101880008B818295807F9C819F70892B8A8384E8DD
:1018900093E00E943B2C89810E94B42C8A810E9493
:1018A000B42C8CE061E0AE014F5F5F4F0E94F425E5
:1018B000882319F084E192E002C080E292E00E9465
:1018C000292C80E00F900F900F900F90DF91CF9117
:1018D0000895CF93DF938FE693E00E943B2CC0E006
:1018E000D0E080E5BE0140E00E94FA24219682E02B
:1018F000C030D807B1F78BE292E00E94292C80E03B
:10190000DF91CF910895EF92FF920F931F93CF93A2
:10191000DF9300D000D000D0CDB7DEB782E392E0F5
:101920000E94292C81E56AEF70E046E050E09E01BC
:101930002F5F3F4F0E945725882329F084E492E0CF
:101940000E94292C10C07E010894E11CF11C00E0CB
:1019500010E0F70181917F010E94B42C0F5F1F4FAF
:1019600006301105B1F782E192E00E94292C80E057
:1019700026960FB6F894DEBF0FBECDBFDF91CF9194
:101980001F910F91FF90EF900895CF93DF9380E028
:101990000E94EA08EC0184E393E00E943B2CBE0124
:1019A00080E090E024E63DE84DE050E00E94572FB3
:1019B0000E946B2C81E00E94EA08EC018FE393E027
:1019C0000E943B2CBE0180E090E022E836E044E03B
:1019D00050E00E94572F0E946B2C82E00E94EA0880
:1019E000EC018FE493E00E943B2CBE0180E090E08C
:1019F0002BEE37E040E050E00E94572F0E946B2C06
:101A000083E00E94EA08EC018FE593E00E943B2C02
:101A1000BE0180E090E020E13AE340E050E00E9427
:101A2000572F0E946B2C8EE492E00E94292C80E0BC
:101A3000DF91CF910895EF92FF920F931F93CF9371
:101A4000DF9300D0CDB7DEB786E293E00E943B2C57
:101A5000CE0101960E949A2290E00E946B2C03E531
:101A600012E0C8010E94292C89819A810E946B2C66
:101A700022E1E22E22E0F22EC7010E94292CCE01A3
:101A800001960E94850B90E00E946B2CC8010E9479
:101A9000292C89819A810E946B2CC7010E94292CD4
:101AA00080E00F900F90DF91CF911F910F91FF90E9
:101AB000EF9008958CE093E00E943B2C86E00E941A
:101AC000292080E008958FEF92E00E943B2C81E076
:101AD0000E94292080E0089582EF92E00E943B2C32
:101AE00080E00E94292080E0089585EE92E00E9427
:101AF0003B2C0E94402490E00E946B2C82E192E0FB
:101B00000E94292C88E00E94292080E00895CF932C
:101B1000DF930F92CDB7DEB788ED92E00E943B2CA9
:101B2000CE01019660E040E050E00E94DC0A90E0C7
:101B30000E946B2C83E592E00E94292C898190E021
:101B40000E946B2C82E192E00E94292C87E00E9487
:101B5000292080E00F90DF91CF910895CF93DF93FC
:101B60000F92CDB7DEB78BEC92E00E943B2CCE01FA
:101B7000019660E040E050E00E94952390E00E94D2
:101B80006B2C83E592E00E94292C898190E00E94D1
:101B90006B2C82E192E00E94292C85E00E94292092
:101BA00080E00F90DF91CF9108958EEE91E00E943A
:101BB0003B2C89EF91E00E943B2C8EE092E00E944A
:101BC0003B2C84E192E00E943B2C84E292E00E9454
:101BD0003B2C8AE292E00E943B2C85E392E00E943B
:101BE0003B2C8EE392E00E943B2C83E492E00E9427
:101BF0003B2C8FE492E00E943B2C83E592E00E9414
:101C00003B2C8CE592E00E943B2C8FE592E00E94F9
:101C10003B2C0E94B60A90E00E946B2C8DE692E06D
:101C20000E943B2C8FE692E00E943B2C0E941120E8
:101C300090E00E946B2C8DE792E00E943B2C80E0AC
:101C4000089585E592E00E94292C10926A04089577
:101C5000CF93DF93AC01A0E08A2F90E0880F991F0B
:101C6000880F991FFC01EF53FD4F60817181B0E037
:101C70002B2F30E0FB01E20FF31FE081EE2359F040
:101C8000240F351FE90128812E272F7511F4BF5F1E
:101C9000EFCFAF5FE1CFBB2349F08F539D4FDC0106
:101CA0001296ED91FC911397099501C081E0DF91A7
:101CB000CF910895CF93DF930F92CDB7DEB7CE01CA
:101CC00001960E94AF2B882309F04CC0898188308F
:101CD00019F08D3081F510C080916A04882309F4D1
:101CE00041C0815080936A0488E00E94902B80E27A
:101CF0000E94902B88E034C08AE00E94902B8DE0F7
:101D00000E94902BE0916A04EE2371F0F0E0E55917
:101D1000FB4F10828BE694E00E94280E882321F06E
:101D20008FE592E00E94292C10926A0480E792E0ED
:101D30000E94292C17C08B31A9F090916A0490322F
:101D400070F40E94902B80916A04E82FF0E0E5592E
:101D5000FB4F998190838F5F80936A0403C087E073
:101D60000E94902B0F90DF91CF9108950F931F93B6
:101D7000CF93DF93C7E3D0E0CE010E94D82F90E04D
:101D80008F70907024E630E0829F8001839F100D59
:101D9000929F100D1124CE0101960E94D82F90E041
:101DA0008F7090709C01220F331F53E0880F991F92
:101DB0005A95E1F7280F391F020F131FCE01029623
:101DC0000E94D82F8F709801280F311DC901DF9113
:101DD000CF911F910F910895CF92DF92EF92FF92D2
:101DE0000F931F9387E390E00E94D82F90E08F70AD
:101DF000907024E630E0829F6001839FD00C929F18
:101E0000D00C1124EE24D7FCE094FE2C88E390E063
:101E10000E94D82F90E08F7090709C01220F331F8A
:101E200063E0880F991F6A95E1F7280F391FC901F0
:101E3000AA2797FDA095BA2FC80ED91EEA1EFB1E31
:101E400089E390E00E94D82F8F70A7019601280F98
:101E5000311D411D511DDA01C901529AEFE9FFE020
:101E60003197F1F700C000005298E0E2F0E000E0A6
:101E700010E020E030E8539AB901A8014823592323
:101E80006A237B23411551056105710509F05398BB
:101E9000F894529A52987894369527951795079505
:101EA000319749F71F910F91FF90EF90DF90CF90FE
:101EB000089590E29093B8008E7F8093BA001092BC
:101EC000BD0084E48093BC001092950410929404A9
:101ED0000895CF938091BC0087FF67C0C091B9007F
:101EE000C87FC03661F0C13620F4CC2309F448C065
:101EF00051C0C038D1F0C03A09F04CC02BC010928C
:101F00000904E0911C09F0911D098081806880839B
:101F100080818E7F80838091BB00838381E080936A
:101F2000090494EC9093BC0012C0E0911C09F0915C
:101F30001D09809109049091BB00E80FF11D938366
:101F40008F5F8093090484EC8093BC0081E08093D0
:101F500008042BC0E0911C09F0911D09809109042F
:101F6000828380818160808380818F77808384EC0D
:101F70008093BC00109208048AE080931C0315C073
:101F800081EA93E00E943B2C8091BC0080698093A1
:101F9000BC000BC080EB93E00E943B2C8C2F0E9476
:101FA000B42C81E093E00E94292C80910804CF9109
:101FB0000895CF92DF92FF920F931F93CF93DF93F9
:101FC0000F92CDB7DEB780910704882341F490913A
:101FD000950480919404981709F053C0E5C08F3F91
:101FE00039F484E60E945B2B8EEF80930704DCC0FB
:101FF0008E3F09F046C08091C608882311F14091B8
:10200000940450E023E430E0429FC001439F900DD0
:10201000529F900D11248A569B4F0E94D91F909178
:102020009304891771F4809194048F5F80939404D2
:10203000803111F410929404109207041092C60893
:10204000B3C00E946B2B882309F4AEC080910A04B0
:10205000815080930A04882321F084E60E945B2B40
:1020600010C0809194048F5F80939404803111F4A8
:102070001092940483E093E00E94292C10920704AC
:1020800093C084EA8093BC008091BC0087FFFCCFA2
:102090001091B900187F183059F083EC93E00E943A
:1020A0003B2C812F0E94B42C81E093E00E94292CCC
:1020B0002091940430E083E490E0289FF001299F70
:1020C000F00D389FF00D1124EA56FB4F8381809369
:1020D000BB0084E88093BC008091BC0087FFFCCFEC
:1020E0001091B900187F183159F08DEC93E00E94DF
:1020F0003B2C812F0E94B42C81E093E00E94292C7C
:1021000011E083E4C82ED12C94E8F92E04E923C011
:10211000181719F40093BC001DC0E10FF11D838155
:102120008093BB00F092BC008091BC0087FFFCCF85
:102130002091B900287F283269F087ED93E0298348
:102140000E943B2C2981822F0E94B42C81E093E0D5
:102150000E94292C1F5F20919404822F90E08C9D77
:10216000F0018D9DF00D9C9DF00D1124EA56FB4F62
:102170008281811768F68181813059F4809107044A
:102180008E3F79F08FEF8093070483E080930A04F9
:1021900008C0822F8F5F80939404803111F41092D5
:1021A000940484EC8093BC000F90DF91CF911F9139
:1021B0000F91FF90DF90CF90089560919504462F86
:1021C00050E023E430E0429FF001439FF00D529F26
:1021D000F00D1124EA56FB4FDC0183E40D900192CF
:1021E0008150E1F76F5F60939504603111F41092B4
:1021F000950480E0089591E09093C608809393043D
:102200000895DA01A90190E026E130E0829FF00113
:10221000839FF00D929FF00D1124E953F74F6187D2
:1022200010861286B183A083128213825583448361
:1022300016821782089590E026E130E0829FD00157
:10224000839FB00D929FB00D1124A953B74F662301
:10225000D1F412968C91129790E0880F991FED910E
:10226000FC911197E80FF91F5183408312968C91CE
:1022700012978F5F12968C9312978430F1F4129616
:102280001C921297089516968C91169790E0880FDD
:10229000991F1496ED91FC911597E80FF91F518342
:1022A000408316968C9116978F5F16968C9316978F
:1022B000843019F416961C9216970895CF93DF93E5
:1022C000EA0190E026E130E0829FD001839FB00DCB
:1022D000929FB00D1124A953B74F662309F51396A9
:1022E0008C91139712969C9112978917D9F190E0CF
:1022F000880F991FED91FC911197E80FF91F8081CC
:1023000091819983888313968C9113978F5F13968D
:102310008C931397843041F513961C92139724C025
:1023200017968C91179716969C9116978917D1F04E
:1023300090E0880F991F1496ED91FC911597E80F86
:10234000F91F808191819983888317968C911797C3
:102350008F5F17968C931797843031F417961C92E1
:10236000179702C081E001C080E0DF91CF9108950E
:10237000EF92FF920F931F93CF93DF9300D0CDB7CF
:10238000DEB7F82E282F30E086E190E0289F80010C
:10239000299F100D389F100D11240953174FF80174
:1023A0008085882309F0BCC08285813041F081306E
:1023B00068F0823089F0833009F04BC028C025B125
:1023C000F80191859095922395B942C085B1F801A5
:1023D0009185892B85B93BC0F8018585882349F013
:1023E00095B181858095892385B9858581508587BB
:1023F0000BC0F8018685882339F085B19185892B3A
:1024000085B9868581508687F80186851AC0F801CE
:102410008685882341F085B19185892B85B986858C
:10242000815086870CC0F8018585882341F095B1DD
:1024300081858095892385B9858581508587F801B7
:102440008585882331F4838585878485868781E027
:102450008787F801E784F1E0EF1609F0CEC08F2DF1
:1024600061E0AE014F5F5F4F0E945E11882321F54E
:10247000F801E08649815A81CA019070009711F4F1
:10248000108A4BC09C01215030402A3F310540F456
:1024900082E0F801808B518B428B538B448B3DC083
:1024A0008C3F910519F4F801108637C08F3F9105D4
:1024B000A1F5F801E08A31C08F2D60E0AE014F5FD9
:1024C0005F4F0E945E11882341F589819A81907047
:1024D0008130910551F08130910550F082309105A5
:1024E00051F083309105C9F40FC0F801E28615C0A0
:1024F000F801128612C09AE0F80193878AE5848772
:102500009587868782E008C09AE5F80193878AE07C
:1025100084879587868783E08287F80117866DC058
:10252000F8018089813039F0813060F0823081F0AB
:10253000833081F519C025B1F801918590959223DA
:1025400095B927C085B1F8019185892B85B920C03F
:10255000F8018489882341F085B19185892B85B95B
:1025600084898150848B0CC0F8018389882341F0D1
:1025700095B181858095892385B983898150838B25
:10258000F8018389882331F48189838B8289848B44
:1025900081E0858BF8018589882379F18F2D61E0B1
:1025A000AE014F5F5F4F0E945E11882321F561E00D
:1025B000F801608749815A81CA019070009711F42F
:1025C000108A19C09C01215030402A3F310540F447
:1025D00082E0F801808B518B428B538B448B0BC074
:1025E0008C3F910519F4F801108605C08F3F9105C5
:1025F00011F4F801608BF801158A0F900F90DF91AC
:10260000CF911F910F91FF90EF900895DB0190E023
:1026100026E130E0829FF001839FF00D929FF00D44
:102620001124E953F74F80858C93828511968C9302
:102630001197848512968C931297838513968C93A9
:102640001397808914968C931497828915968C938E
:102650001597818916968C9316970895CF92DF92DD
:10266000EF92FF920F931F93CF93DF930F92CDB70B
:10267000DEB77B0189830E94722A898181600E9472
:10268000952A882321F40E948A2A81E012C081E0E1
:102690000E94CA2A182F00E080E00E94CA2AC82E91
:1026A000DD24C02AD12A0E948A2AF701D182C08261
:1026B00080E00F90DF91CF911F910F91FF90EF90ED
:1026C000DF90CF9008951F920F920FB60F920BB626
:1026D0000F9211242F933F934F935F936F937F93A8
:1026E0008F939F93AF93BF93EF93FF930E94FA2A28
:1026F00080910B0490910C04A0910D04B0910E04F4
:102700000196A11DB11D80930B0490930C04A0931E
:102710000D04B0930E0480910F0490911004019663
:102720009093100480930F0423E0883E920739F4BD
:1027300081E080930C091092100410920F04809194
:1027400011048F5F80931104843629F481E0809313
:102750000D0910921104809112048F5F809312046E
:102760008A3071F40E94712B81E0809319091092D4
:10277000120480912E04882319F0815080932E0436
:10278000FF91EF91BF91AF919F918F917F916F9149
:102790005F914F913F912F910F900BBE0F900FBE05
:1027A0000F901F90189585B1817F85B9209A289840
:1027B0008FEC97E00197F1F700C0000021E0199B32
:1027C00020E081E01A9B80E091E01B9B90E0289A3A
:1027D000EFECF7E03197F1F700C0000063B141E0A2
:1027E0001A9B40E031E01B9B30E051E061FF50E07C
:1027F000251322E0841382E0931392E0E82FEE0F7A
:10280000E80FE20F89E0989F902D1124E90FF0E086
:10281000E05CFA4F8491089590E08057904062E028
:1028200070E00E94822F862F0895FC018481869596
:10283000869581700895FC0183819481890F81952B
:1028400085838281DF0123E090E005C015963C91ED
:102850001597930F2F5F11962817C0F3DF01A80F6C
:10286000B11D919513969C9313978F5F8283089562
:10287000CF93DF93EC0188818E7F806888830E94EC
:10288000D90F88818F77888380E0DF91CF91089579
:10289000FC0183819481890F819595819817D9F4E2
:1028A000828190E0019753E040E008C02E0F3F1F67
:1028B000D90113962C911397420F5F5F252F30E0BB
:1028C000281739079CF3E80FF91F41958381841776
:1028D00021F082E0089581E0089580E008959F92BC
:1028E000AF92BF92CF92DF92EF92FF920F931F931E
:1028F000CF93DF93CDB7DEB760970FB6F894DEBF06
:102900000FBECDBF8C017B01FE013296AEE5B3E078
:1029100086E00D9001928150E1F7D80114962C9138
:102920001497269526952A3009F447C32B3040F496
:10293000243009F44FC0263011F00C94951F09C0C3
:102940002C3209F48FC4203311F00C94951F0C9491
:102950002A1DF8018085813011F00C94951F8EECB2
:1029600097E00E943B2CD80116968C911697F701A0
:10297000838317969C91179714968C9114978C5F6C
:102980008C7F292F2370822B848380911709868363
:1029900014968C91149783709C7F892B878318964B
:1029A0008C91189780871186128681E8838782E050
:1029B000848785E7858781E586878BE287878DEB2E
:1029C000808B82E9818B128A138A83E8848B82E16F
:1029D0000C94D41FD80118968C911897803209F462
:1029E0009FC0813248F4813009F446C0813088F0BC
:1029F000823009F0D9C26EC0823209F45EC18232DF
:102A000008F4BDC0873209F41AC28D3209F0CCC275
:102A100084C182EF97E00E943B2CF801818580936E
:102A200062098285809363098681D70113968C930E
:102A30001397978184818C5F8C7F292F2370822B41
:102A400014968C9314978091170916968C93169769
:102A5000848183709C7F892B17968C931797808530
:102A600018968C93189719961C920E94D80A0E9467
:102A7000252087E00C94AE1E82E298E00E943B2C59
:102A8000D80116968C911697F701838317969C911F
:102A9000179714968C9114978C5F8C7F292F237035
:102AA000822B848380911709868314968C911497C6
:102AB00083709C7F892B878318968C9118978087C9
:102AC000118680916209828780916309838789E0FA
:102AD0000C94D41F82E598E00E943B2CD8011696F6
:102AE0008C911697F701838317969C9117971496EC
:102AF0008C9114978C5F8C7F292F2370822B848379
:102B000080911709868314968C91149783709C7F0B
:102B1000892B878318968C91189780871186FBC222
:102B20008EE798E00E943B2CD80116968C91169760
:102B3000F701838317969C91179714968C9114979D
:102B40008C5F8C7F292F2370822B848380911709BF
:102B5000868314968C91149783709C7F892B87832E
:102B600018968C91808711860E945A2AD7011A964E
:102B70008C931A9781E01B968C931B97CCC08FEA9D
:102B800098E00E943B2CF8018681D70113968C9324
:102B90001397978184818C5F8C7F292F2370822BE0
:102BA00014968C9314978091170916968C93169708
:102BB000848183709C7F892B17968C9317978085CF
:102BC00018968C93189719961C92A384BB2494850D
:102BD00080E0A82AB92AC58496840E945A2A0197BF
:102BE000A816B90629F48FEFF7018287838708C0FA
:102BF000C5010196D7011A968C931A971B969C9340
:102C0000F501EE0FFF1FEC59FC4F0C2D10E0608119
:102C10007181600F711FC7010C96492D50E00E9411
:102C2000A92FB5E0BC1560F0C801890D911D853054
:102C3000910534F0F701E01BF10B80911709818BAE
:102C4000E2E0AE16B104C8F4FDE0FC1570F1DD243D
:102C5000C601890D911D8D3091053CF1F701EC19EC
:102C6000FD098091170990E08057904062E070E084
:102C70000E94822F605A618F18C049E04C15A8F05D
:102C8000DD24C601890D911D8930910574F0F7018D
:102C9000EC19FD098091170990E08057904062E09F
:102CA00070E00E94822F605A658B892D875FD70163
:102CB00012968C9312970C94B81F8BED98E00E949B
:102CC0003B2CF8018681D70113968C93139797813B
:102CD00084818C5F8C7F292F2370822B14968C9398
:102CE00014978091170916968C9316978481837098
:102CF0009C7F892B17968C931797808518968C93B9
:102D0000189719961C92199781E01A968C931A9726
:102D10001B961C921B9789E0CBCF8BE099E00E9419
:102D20003B2CF8018681D70113968C9313979781DA
:102D300084818C5F8C7F292F2370822B14968C9337
:102D400014978091170916968C9316978481837037
:102D50009C7F892B17968C931797808518968C9358
:102D6000189719961C92199781859AE012969C9350
:102D700012978430C9F1853058F4813009F18130DF
:102D800098F0823001F1833011F00C94B81F1EC00E
:102D9000863009F43FC08630D8F18730E9F18830B9
:102DA00011F00C94B81F48C0F701128680EC83879D
:102DB0000E94B90AD7011C968C931C970C94B81FDB
:102DC00080910A090AC08091100915C080E00E9414
:102DD000EA089695879596958795F701828780E40E
:102DE000838714860C94B81F81E00E94EA089695A8
:102DF000879596958795D7011A968C931A9780E4B4
:102E00001B968C931B971C961C921C970C94B81FB6
:102E100082E0DDCF83E0E9CFF701128680EC838783
:102E20000E941420D7011C968C930E941420F70155
:102E300095878BE00C94D41F80911B09DCCF8BE32A
:102E400099E00E943B2CF8018681D70113968C9360
:102E50001397978184818C5F8C7F292F2370822B1D
:102E600014968C9314978091170916968C93169745
:102E7000848183709C7F892B17968C93179780850C
:102E800018968C93189719961C92199781858430FF
:102E900009F43CC0853050F48130B9F0813090F0B5
:102EA0008230E9F0833009F07DC026C0863009F415
:102EB00041C08630A8F1873009F474C0883009F029
:102EC00071C042C0F7010C94D21F8FE3D7011A964C
:102ED0008C931A9780916A0390916B0309C08FE3DA
:102EE000D7011A968C931A9780916C0390916D0379
:102EF000FC01B996E49133C08FE3D7011A968C9305
:102F00001A9780916E0390916F03F2CF8FE3D701F0
:102F10001A968C931A978091700390917103E8CF61
:102F20008FE3D7011A968C931A9780917203909130
:102F30007303DECF8FE3D7011A968C931A97809193
:102F4000740390917503D4CF8FE3F701828780914A
:102F5000780390917903FC01B996E491D7011B960F
:102F6000EC931B97FC01B896E4911C96EC931C978C
:102F7000FC01B796E4911D96EC931D97FC01B69663
:102F8000E4911E96EC931E97FC01B596E4911F9672
:102F9000EC931F978496FC01849150968C935097E4
:102FA0008EE086CED7011EC48EE699E00E943B2CAF
:102FB000F80180850E94B42C48C5D80118968C91E0
:102FC0001897813109F452C0823109F4B2C08031BE
:102FD00009F0ABC780E999E0288B0E943B2CF801EF
:102FE00081852889882351F08130D1F4288B0E9473
:102FF00011202889882311F483ED13C0D7011A9674
:103000001C921A9782E01B968C931B971C961C921D
:103010001C9719961C92199712962C93129705C01B
:1030200089ECF701818787E08283D80116968C911D
:103030001697F701838317969C91179714968C9196
:1030400014978C5F8C7F292F2370822B848380912F
:103050001709868314968C91149783709C7F892B13
:10306000878318968C911897808782C780EC99E0A7
:103070000E943B2CD80116968C911697F7018383FA
:1030800017969C91179714968C9114978C5F8C7F50
:10309000292F2370822B84838091170986831496AD
:1030A0008C91149783709C7F892B878318968C91C1
:1030B0001897808711861A96AC901A97BB241B9696
:1030C0009C911B9780E0A82AB92A1C96CC901C974B
:1030D000C28619968C911997882321F0813009F0C6
:1030E00047C70EC089EE99E00E943B2CB5016050A5
:1030F0007040C7010B964C2D50E00E94C82F16C09F
:103100008EEE99E00E943B2C0E941120882329F426
:1031100083EDF701818787E047C79701255F3F4F20
:1031200080E5B5014C2D50E00E943D228C2D885F3A
:10313000BECD83EF99E00E943B2CF801C280F6EFF0
:10314000CF0ED8011A96AC901A97BB241B969C916F
:103150001B9780E0A82AB92A19968C911997882381
:1031600021F0813009F05DC014C08DE19AE00E9429
:103170003B2CF701C286B50160507040C8010C9627
:103180004C2D50E00E94E02FD70119961C92199700
:1031900048C082E29AE00E943B2C80E593E00E94C6
:1031A000292CC5010E946B2C86E593E00E94292CF6
:1031B0008C2D90E00E946B2C8EE493E00E94292CD1
:1031C0000E941120F701882349F1C28611868CE7FD
:1031D000BE016F5F7F4F0E949B208823B1F46981FD
:1031E00061616F7769838CE70E94C020882311F0AA
:1031F000F70114C09801245F3F4F80E5B5014C2DC5
:1032000050E00E942F25882361F0D7011A961C9266
:103210001A9783ED19968C93199703C0128683ED44
:103220008187D80116968C911697F701838317969C
:103230009C91179714968C9114978C5F8C7F292FF3
:103240002370822B848380911709868314968C9136
:10325000149783709C7F892B878318968C9118977D
:103260008087A1C6D80118968C9118978C3009F4E4
:1032700068C38D30A8F4853009F4B7C0863030F4C7
:10328000882321F1843009F0C8C357C0873009F47E
:10329000E2C0873008F4DCC0883009F0BEC361C1E9
:1032A000893109F415C38A3138F48D3009F4C3C269
:1032B000813109F0B2C375C38E3109F406C38D3272
:1032C00009F43CC38A3109F0A8C335C387E29AE008
:1032D0000E943B2CF8018681D70113968C9313979B
:1032E000978184818C5F8C7F292F2370822B149689
:1032F0008C9314978091170916968C931697848156
:1033000083709C7F892B17968C93179780851896CE
:103310008C93189719961C9219971A961C921A97C3
:1033200082E31B968C931B9781E01C968C931C97D1
:103330001D961C921D978BE0BBCC8FE49AE00E94F7
:103340003B2CF8018681D70113968C9313979781B4
:1033500084818C5F8C7F292F2370822B14968C9311
:1033600014978091170916968C9316978481837011
:103370009C7F892B17968C931797808518968C9332
:10338000189719961C9219971A961C921A9788E00A
:1033900012968C9312978285882321F0813009F050
:1033A000FEC515C084E79AE00E943B2CF801838596
:1033B000882321F0843009F0F2C506C01092160966
:1033C00082E30E94402BD4C50E94D00AD1C589E770
:1033D0009AE00E943B2CD8011B968C911B9784305D
:1033E00009F0DDC50E942120C3C58EE79AE00E9446
:1033F0003B2CF8018681D70113968C931397978104
:1034000084818C5F8C7F292F2370822B14968C9360
:1034100014978091170916968C9316978481837060
:103420009C7F892B17968C931797808518968C9381
:10343000189719961C9219971A961C921A9787E05A
:103440001B968C931B971C961C921C978AE030CC81
:1034500088EA9AE068C584ED9AE00E943B2CF80166
:10346000248545858285882321F0813009F041C279
:1034700027C0C22EDD24942F80E0C82AD92A838554
:103480008130B1F0813020F0823009F087C112C064
:1034900080E061E0A6010E941B110E94B60A823002
:1034A00009F027C2CC2009F024C20E94BC0A21C224
:1034B00081E001C082E061E0A6010E941B1119C2F7
:1034C000F8018385813081F0813018F0823049F530
:1034D00016C0222319F02F3F29F402C080E015C046
:1034E00080E01AC080E01BC0222319F02F3F29F48E
:1034F00002C081E00AC081E00FC081E010C0222339
:1035000019F02F3F59F407C082E060E040E020E06E
:103510000E94DE1FEEC182E061E0F8CF82E062E04F
:10352000F7CFD8018681F701838317969C9117976F
:1035300014968C9114978C5F8C7F292F2370822B8B
:10354000848380911709868314968C9114978370D5
:103550009C7F892B878318968C91189780878CEC99
:1035600020C58EEF9AE00E943B2C19820DC0F80115
:10357000E80FF11D83810E94B42C8CE593E00E943A
:10358000292C89818F5F89838981D80112969C912A
:103590001297891760F38EE493E00E94292CF801BA
:1035A0008285882309F023C18385813009F44FC0C7
:1035B000813020F0823009F0E4C08FC080E0BE018D
:1035C000685F7F4F0E9406138985882319F0813038
:1035D00071F404C0F701148615860EC08FEFD70171
:1035E0001C968C931C971D961C921D9705C08A856E
:1035F000F70184878B85858781E0D7011E968C93A0
:103600001E979CE012969C9312979885913009F032
:10361000B5C082E01B968C931B978C85882319F08C
:10362000813071F404C0F7011786108A0EC08FEF45
:10363000D7011F968C931F9750961C92509705C0E8
:103640008D85F70187878E85808B81E08DC081E035
:10365000BE01685F7F4F0E9406138985882319F099
:10366000813071F408C0D7011C961C921C971D96DE
:103670001C921D970EC08FEFF7018487158609C035
:103680008A85D7011C968C931C978B851D968C93ED
:103690001D9782E0F70186879CE0928398859130A0
:1036A000C9F483878C85882319F0813049F403C0DD
:1036B0001786108A09C08FEFF7018787108A04C028
:1036C0008D8587878E85808B82E0F701818B8FE0E7
:1036D00082838DC081E083878AC082E0BE01685FFB
:1036E0007F4F0E9406138985882319F0813071F479
:1036F00004C0F701148615860EC08FEFD7011C9603
:103700008C931C971D961C921D9705C08A85F70106
:1037100084878B85858783E0D7011E968C931E97BF
:103720008CE012968C9312978885813031F582E077
:103730001B968C931B978C85882319F0813071F42C
:1037400004C0F7011786108A0EC08FEFD7011F96AD
:103750008C931F9750961C92509705C08D85F7014A
:1037600087878E85808B83E0D70151968C93519704
:103770008FE012968C9312973AC081E0F70183870D
:1037800036C088E29BE00E943B2CD8011A968C91AF
:103790000E94B42C86E59BE00E943B2CF8018681B8
:1037A000D70113968C931397978184818C5F8C7FBC
:1037B000292F2370822B14968C93149780911709CC
:1037C00016968C931697848183709C7F892B17960D
:1037D0008C931797808518968C9318978CEC199674
:1037E0008C9319971A961C921A9788E061CAF8016F
:1037F0008681D70113968C931397978184818C5F70
:103800008C7F292F2370822B14968C931497809190
:10381000170916968C931697848183709C7F892B49
:1038200017968C931797808518968C9318971996EE
:103830001C92199746C088E59BE00E943B2CF8013A
:103840008285882319F08130A1F40CC0D7011B9622
:103850001C921B971C961C921C9719961C921997E8
:103860008AE00DC0F7018387148611868AE082837F
:1038700008C08CECD70119968C93199787E01296A3
:103880008C93F8018681D70113968C9313979781B7
:1038900084818C5F8C7F292F2370822B14968C93CC
:1038A00014978091170916968C93169784818370CC
:1038B0009C7F892B17968C931797808518968C93ED
:1038C00018971A961C921A9753C385E89BE02BC34E
:1038D0008FEA9BE00E943B2CF8018685882319F033
:1038E0000E94C00A06C00E94B60A853011F40E94E8
:1038F000C80AD80116968C911697F70183831796FC
:103900009C91179714968C9114978C5F8C7F292F1C
:103910002370822B848380911709868314968C915F
:10392000149783709C7F892B878318968C911897A6
:103930008087118637C38AED9BE0F5C285E09CE065
:10394000F2C28DE29CE00E943B2CD80116968C912D
:103950001697F701838317969C91179714968C916D
:1039600014978C5F8C7F292F2370822B8483809106
:103970001709868314968C91149783709C7F892BEA
:10398000878318968C9118978087128688E08283A7
:103990001A968C911A978823A1F1813009F0E8C218
:1039A00019C188E59CE00E943B2CD80116968C91A9
:1039B0001697F701838317969C91179714968C910D
:1039C00014978C5F8C7F292F2370822B84838091A6
:1039D0001709868314968C91149783709C7F892B8A
:1039E000878318968C9118978087128688E0828347
:1039F0001A968C911A97882321F0813009F0B8C269
:103A000002C08FEF14C1F8018385882319F00E944A
:103A100019207FC20E941D207CC280E89CE00E9489
:103A20003B2C19820DC0F801E80FF11D83810E9423
:103A3000B42C8CE593E00E94292C89818F5F8983C7
:103A40008981F8019281891770F38EE493E00E94D6
:103A5000292C6BC2D80118962C911897253009F49F
:103A60000AC1263060F42130B9F0213008F437C1A2
:103A7000223009F462C0233009F053C2AEC02730AF
:103A800009F4A3C1273008F46BC1283009F4DCC164
:103A9000293009F046C20EC28CE99CE00E943B2C02
:103AA000F801C1849284D384A4848681D7011396BB
:103AB0008C931397978184818C5F8C7F292F23703F
:103AC000822B14968C9314978091170916968C93D9
:103AD0001697848183709C7F892B17968C931797F8
:103AE000808518968C93189787E012968C93B0E196
:103AF000BA1510F482E813C20E941120882309F439
:103B000095C0CC2011F490E5C92E692D70E09D2D53
:103B100080E0682B792B9701265F3F4F8C2D4A2D33
:103B200050E00E943D22882309F0A3C0D7011996D6
:103B30001C9219978A2D895FBBC881EC9CE00E947A
:103B40003B2CF801C184A284D38444858681D701AB
:103B500013968C931397978184818C5F8C7F292F88
:103B60002370822B14968C931497809117091696C4
:103B70008C931697848183709C7F892B17968C93E6
:103B80001797808518968C93189787E012968C93D8
:103B90001297413110F082E84BC0488B0E941120EF
:103BA0004889882311F480E8BAC1CC2011F480E55B
:103BB000C82E6A2D70E09D2D80E0682B792B98012E
:103BC000235F3F4F8C2D50E00E942F25882311F05A
:103BD00081E82DC0F7011186CBC187EE9CE00E94E1
:103BE0003B2CD80116968C911697F7018383179674
:103BF0009C91179714968C9114978C5F8C7F292F2A
:103C00002370822B848380911709868314968C916C
:103C1000149783709C7F892B878318968C9180875B
:103C200087E082830E941120882331F480E8D70145
:103C300019968C9319979CC18CE7BE016F5F7F4FDB
:103C40000E949B208823A9F48981982F9161D80133
:103C500019962C911997222311F0816902C0892F9E
:103C60008F7789838CE769810E94C020882309F4BB
:103C700050C181E854C181E19DE00E943B2CF801D4
:103C80008681D70113968C931397978184818C5FDB
:103C90008C7F292F2370822B14968C9314978091FC
:103CA000170916968C931697848183709C7F892BB5
:103CB00017968C931797808518968C93189787E0A2
:103CC00012968C931297389A8FEF99E6A8E181505B
:103CD0009040A040E1F700C0000038981AC185E389
:103CE0009DE00E943B2CF8018681D70113968C93AE
:103CF0001397978184818C5F8C7F292F2370822B6F
:103D000014968C9314978091170916968C93169796
:103D1000848183709C7F892B17968C93179780855D
:103D200018968C93189787E012968C931297199691
:103D30001C92199720E00FC0822F90E0F701E80F46
:103D4000F91F42E050E04C0F5D1F840F951FDC010E
:103D50008C9182872F5F253078F38CE0F70124C1A6
:103D600080E69DE00E943B2CD80116968C91169718
:103D7000F701838317969C91179714968C9114974B
:103D80008C5F8C7F292F2370822B8483809117096D
:103D9000868314968C91149783709C7F892B8783DC
:103DA00018968C911897808787E082838DEC8187A5
:103DB00080911304882309F4DBC0A701465F5F4F9D
:103DC0008CE061E00E941C296AC08CE89DE0288B91
:103DD0000E943B2CD80119968C91199780936C09FD
:103DE0001A968C911A9780936D0916968C91169756
:103DF000F701838317969C91179714968C911497CB
:103E00008C5F8C7F392F3370832B848380911709CB
:103E1000868314968C91149783709C7F892B87835B
:103E200018968C9118978087288922838DEC81873A
:103E300080911304882309F49BC08CE061E04CE678
:103E400059E00E94F42563C088EB9DE00E943B2C62
:103E5000D80116968C911697F701838317969C913B
:103E6000179714968C9114978C5F8C7F292F237051
:103E7000822B848380911709868314968C911497E2
:103E800083709C7F892B878318968C91808787E02D
:103E90008283B7016F5E7F4F88E40E947E2988236A
:103EA000E9F5D70112968C9112978E5F12968C933A
:103EB000129730C085EE9DE00E943B2CD8011996E8
:103EC0006C91199760936C0916968C911697F7016F
:103ED000838317969C91179714968C9114978C5FF7
:103EE0008C7F292F2370822B8483809117098683EE
:103EF00014968C91149783709C7F892B87831896D6
:103F00008C91808787E0828388E40E9457298823E8
:103F100029F4D70119961C9219972AC08FEFF7013F
:103F200026C080E19EE00E943B2CD80116968C9121
:103F30001697F701838317969C91179714968C9187
:103F400014978C5F8C7F292F2370822B8483809120
:103F50001709868314968C91149783709C7F892B04
:103F6000878318968C91808787E0828381EC818794
:103F7000D70111961C92119781E060960FB6F894C4
:103F8000DEBF0FBECDBFDF91CF911F910F91FF908C
:103F9000EF90DF90CF90BF90AF909F9008958CEC02
:103FA000F7018187128688E08283E2CF8EE199E073
:103FB0000895FC018781869586950895982F842F12
:103FC000913099F0913018F0923051F51CC0609307
:103FD00065093AE0632F0E94762F80936B09822F48
:103FE0000E94762F80936709089560936A093AE0EA
:103FF000632F0E94762F80937009822F0E94762F64
:10400000809369090895609364093AE0632F0E94E0
:10401000762F80936F09822F0E94762F80938109DB
:1040200008958091E003089580911B0490911C04F1
:10403000089581E080931A04089581E08093190423
:10404000089581E080931804089581E08093160418
:1040500008951F93CF93DF93CDB7DEB7C354D040FD
:104060000FB6F894DEBF0FBECDBF182F87E990E1E1
:104070000E943B2C812F0E94B42C8AE793E00E947F
:10408000292C809162098C8380E18D8380911709AE
:104090008F838091610988878C5F8093610982E0BA
:1040A000898784E08A8782EF8B8787E08C878FE619
:1040B0008D871E878BE08B83CE0101960E941B1497
:1040C00081E08A83CE0101960E94DD101093DE0309
:1040D000CD5BDF4F0FB6F894DEBF0FBECDBFDF91D3
:1040E000CF911F91089580916609982F917080FD5E
:1040F00008C080912704882321F01092270481E0D2
:1041000008959093270480E0089580916609982F80
:10411000917080FF08C080912804813021F081E0F7
:104120008093280408959093280480E00895909146
:104130006609892308950F931F93CF93DF930F92FE
:10414000CDB7DEB78B0189830E94CF298981816039
:104150000E94F229882321F40E94E72981E00AC005
:1041600080E00E94282A89830E94E7298981F8013A
:10417000808380E00F90DF91CF911F910F91089580
:104180001F93CF93DF9300D0CDB7DEB76A838983C7
:104190000E94CF2989810E94F2296A81882321F413
:1041A0000E94E72981E009C0862F0E94F229182F7A
:1041B0000E94E72981E0111180E00F900F90DF91BC
:1041C000CF911F9108951F93CF93DF930F92CDB797
:1041D000DEB780916509813029F08130E0F08230CE
:1041E000F1F405C010921F041092200409C08091C0
:1041F0001F0490916B09891728F48F5F80931F0427
:1042000011E00EC0809120048F5F80932004909174
:104210006709891721F410921F041092200410E0FE
:1042200080916A09813029F08130F0F0823001F507
:1042300006C01092210410922204126019C012606C
:104240008091210490917009891720F48F5F8093E9
:1042500021040EC01D7F809122048F5F8093220471
:1042600090916909891721F4109221041092220477
:1042700080916409813029F08130F0F0823001F5BD
:1042800006C01092230410922404146019C0146014
:104290008091230490916F09891720F48F5F809398
:1042A00023040EC01B7F809124048F5F809324041D
:1042B00090918109891721F410922304109224040B
:1042C0008091E003882351F18CE7BE016F5F7F4F3F
:1042D0000E949B20882311F581E080931D04898131
:1042E000809366098F61898310FF02C08D7F898367
:1042F00011FF03C089818B7F898312FF03C08981ED
:10430000877F898380911404882321F0880F998105
:10431000892789838CE769810E94C0200F90DF91F3
:10432000CF911F9108951F93CF93DF9300D0CDB706
:10433000DEB7162F8CE7BE016F5F7F4F4A830E9466
:104340009B204A81882381F4642F61236161409519
:1043500089814823642B69838CE70E94C02091E007
:10436000882319F490E001C091E0892F0F900F90FD
:10437000DF91CF911F9108951F93CF93DF930F92F9
:10438000CDB7DEB789830E94CF2989810E94F229A7
:10439000882329F089E00E94F229882321F40E94D1
:1043A000E72981E009C080E00E94F229182F0E94CD
:1043B000E72981E0111180E00F90DF91CF911F91EB
:1043C0000895CF92DF92EF92FF920F931F93CF93B6
:1043D000DF930F92CDB7DEB7F82E8B016A010E94F2
:1043E000CF298F2D0E94F229882379F080E00E9446
:1043F000F229882351F00E94DA29EE24E394EF2871
:104400008E2D0E94F229882321F40E94E72981E061
:104410002AC080E00E94282A89830E94E729898196
:10442000F80180830E94CF298F2D0E94F2298823D2
:1044300061F081E00E94F229882339F00E94DA2994
:104440008E2D0E94F229882321F40E94E72982E020
:104450000AC080E00E94282A89830E94E729898176
:10446000F601808380E00F90DF91CF911F910F9133
:10447000FF90EF90DF90CF900895AF92BF92CF92D0
:10448000DF92EF92FF920F931F93CF93DF930F92E0
:10449000CDB7DEB7182F062F6A01E22EA32E79833F
:1044A0000E94CF29812F880F0E94F22979818823C9
:1044B00091F1872F0E94F229882369F1802F0E94B1
:1044C000F229882341F10E94DA29812F880F816027
:1044D0000E94F2298823F9F00E2D1A2DEE24FF24D4
:1044E00056010894A108B1080FC0EA14FB0411F4A6
:1044F00080E001C081E00E94282AF80180830894AE
:10450000E11CF11C0F5F1F4FEC14FD0471F70E94BA
:10451000E72980E003C00E94E72981E00F90DF9146
:10452000CF911F910F91FF90EF90DF90CF90BF90B0
:10453000AF900895EF92FF920F931F93CF93DF9365
:10454000CDB7DEB728970FB6F894DEBF0FBECDBF4C
:104550007C0180E560E070E048E050E09E012F5F64
:104560003F4F0E943D22882309F044C0FE0131964E
:1045700097E02191820F9150E1F7819598858917F5
:1045800031F08CE793E00E94292C82E034C00E8148
:1045900010E083E0000F111F8A95E1F70115110566
:1045A00039F180E5B80145E050E09E012F5F3F4FB3
:1045B0000E943D228823F1F42A819981920F8B81F8
:1045C000980F3C81930F91953D81931731F082E9CB
:1045D00093E00E94292C84E00EC090E00596080F1D
:1045E000191F27FFDECFF7011183008380E003C08E
:1045F00083E001C081E028960FB6F894DEBF0FBEBD
:10460000CDBFDF91CF911F910F91FF90EF90089553
:10461000BF92CF92DF92EF92FF920F931F93CF93AF
:10462000DF93CDB7DEB72A970FB6F894DEBF0FBE83
:10463000CDBF1092130410921404882309F060C0B7
:1046400080E560E070E048E050E06E010894C11C35
:10465000D11C96010E943D22882309F055C00C818F
:1046600010E023E0000F111F2A95E1F70115110555
:1046700009F448C080E5B80147E050E096010E9487
:104680003D22882309F040C08F818F73B801680FE5
:10469000711D685F7F4F80E54AE050E096010E94FF
:1046A0003D22882389F50EEC13E0EE24FF24BC2C78
:1046B000CD2CF8013297D8014C91808191816B2DDE
:1046C0007C2D50E00E94B22F009779F481E0809316
:1046D0001304F701EE0FFF1FEE0FFF1FE453FC4F13
:1046E00083818093140480E010C00894E11CF11CC5
:1046F0000C5F1F4FB3E0EB16F104D9F684E005C060
:1047000082E003C083E001C081E02A960FB6F894EE
:10471000DEBF0FBECDBFDF91CF911F910F91FF90F4
:10472000EF90DF90CF90BF9008959F92AF92BF928D
:10473000CF92DF92EF92FF920F931F93CF93DF936D
:10474000CDB7DEB7C850D1400FB6F894DEBF0FBE6C
:10475000CDBF6C01962E5A01FC01108280E560E00D
:1047600070E048E050E09E012F5F3F4F0E943D22E5
:10477000882309F06DC0FE01319697E02191820FE8
:104780009150E1F781959885891709F05BC00E81FA
:1047900010E033E0000F111F3A95E1F70115110504
:1047A00009F452C080E5B80145E050E09E012F5F5A
:1047B0003F4F0E943D22882309F04AC08A81998197
:1047C000890FEB808E0D9C81890F81959D818917C2
:1047D000E9F5FF240B5F1F4F80E5B801A7019E019B
:1047E000275F3F4F0E943D22882391F590E00AC049
:1047F00049E050E04C0F5D1F240F351FF901208167
:10480000920F8F5F282F30E02E153F0588F391958A
:104810008C819817F9F4F60180818F5F8083891568
:1048200059F4A114B10441F0F501DE0119968DE0AF
:104830000D9001928150E1F78A8187FD0DC00E0D28
:104840001F1DB0CF82E009C083E007C084E005C02F
:1048500081E003C085E001C080E0C85FDE4F0FB695
:10486000F894DEBF0FBECDBFDF91CF911F910F91A6
:10487000FF90EF90DF90CF90BF90AF909F90089502
:104880009F92AF92BF92CF92DF92EF92FF920F93DF
:104890001F93CF93DF93CDB7DEB76D970FB6F89424
:1048A000DEBF0FBECDBF72E0E72EF12CEC0EFD1E79
:1048B000C70160E040E050E00E94DC0A6E0108940D
:1048C000C11CD11CC60160E040E050E00E9495236D
:1048D0008A81882319F480E590E106C089818823C4
:1048E00009F069C089E690E10E943B2C21E06FC08D
:1048F000892D9A2D612FAE01405F5F4F0E94DC0A27
:1049000082E890E10E943B2C60E1E62EF12CEC0E57
:10491000FD1E0DE0F70181917F010E94B42C8FEA0A
:1049200093E00E94292C0150A9F78AE793E00E94A6
:10493000292C21E001E03AC08B2D9C2D602FAE0187
:104940004D5F5F4F2D8F0E9495238E812D8D80337B
:1049500061F5222351F18DE890E10E943B2C43E068
:10496000E42EF12CEC0EFD1E20E0F70181917F0179
:104970002D8F0E94B42C8FEA93E00E94292C2D8D5C
:104980002F5F2D3091F78AE793E00E94292CCE010A
:104990004396BE016A5F7F4F4AE050E00E94B22F0B
:1049A000009711F021E001C020E00F5F898180179E
:1049B00018F61F5F06C021E011E09E2CAF2CBC2C26
:1049C000CD2C8A81811718F0222309F091CF822FF4
:1049D0006D960FB6F894DEBF0FBECDBFDF91CF91BD
:1049E0001F910F91FF90EF90DF90CF90BF90AF900D
:1049F0009F9008950F931F93CF93DF9300D0CDB76F
:104A0000DEB7062F142F7A8389830E94CF298981EC
:104A1000880F0E94F2297A81882351F0872F0E9403
:104A2000F229882329F0802F0E94F229882321F47B
:104A30000E94E72981E00CC0812F0E94F2290E9488
:104A4000E7298FE097E20197F1F700C0000080E0CE
:104A50000F900F90DF91CF911F910F910895AF921A
:104A6000BF92CF92DF92EF92FF921F93CF93DF938B
:104A7000182F6B015A017901C0E0D0E00AC0F7019C
:104A800041917F01BE016C0D7D1D812F0E94FA2492
:104A90002196CA15DB0599F780E0DF91CF911F9130
:104AA000FF90EF90DF90CF90BF90AF900895AF92BE
:104AB000BF92CF92DF92EF92FF920F931F93CF930B
:104AC000DF930F92CDB7DEB7082F6A01E22EA32E37
:104AD00069830E94CF29802F880F0E94F229698163
:104AE0008823B9F0862F0E94F229882391F00E9432
:104AF000DA29802F880F81600E94F229882349F0EB
:104B00000E2D1A2DEE24FF2456010894A108B10899
:104B100013C00E94E72981E015C0EA14FB0411F4D8
:104B200080E001C081E00E94282AF8018083089477
:104B3000E11CF11C0F5F1F4FEC14FD0471F70E9484
:104B4000E72980E00F90DF91CF911F910F91FF90A7
:104B5000EF90DF90CF90BF90AF900895CF92DF920B
:104B6000EF92FF920F931F93CF93DF9300D0CDB7B7
:104B7000DEB77A0169016A8389830E94CF2989811E
:104B8000880F0E94F2296A81882381F0862F0E9473
:104B9000F229882359F08601CC24DD240EC0F801C7
:104BA00081918F010E94F229882321F40E94E72934
:104BB00081E00FC00894C11CD11CCE14DF0479F72A
:104BC0000E94E7298FE097E20197F1F700C000000B
:104BD00080E00F900F90DF91CF911F910F91FF9088
:104BE000EF90DF90CF9008950F931F93CF93DF93B3
:104BF00000D0CDB7DEB78A016A8389830E94CF29AE
:104C00008981880F0E94F2296A818823E1F0862F2A
:104C100083700E94F2298823B1F0F80180810E94FC
:104C2000F229882381F0F80181810E94F2298823EA
:104C300051F00E94E7298FE097E20197F1F700C059
:104C4000000080E003C00E94E72981E00F900F90F0
:104C5000DF91CF911F910F910895CF92DF92EF9244
:104C6000FF928091E0038093DF0320911E04209344
:104C7000E00380911D04882389F0309166098091BA
:104C80001B0490911C0430FD03C08D7F816002C025
:104C900082608E7F90931C0480931B04233009F460
:104CA00074C1243048F48091DF03213009F4AEC090
:104CB000223008F030C10DC0253009F4F4C1253090
:104CC00008F46DC1263009F43DC22B3009F067C2EB
:104CD0006DC08823A9F180E490E090931C04809338
:104CE0001B0487B18F7687B9429A46988AE29EE084
:104CF0000E943B2C87E39EE00E943B2C80911C0489
:104D00000E94B42C80911B040E94B42C8AE793E08B
:104D10000E94292C0E94682A1092250480E060E0FD
:104D200040E020E00E94DE1F81E060E040E020E003
:104D30000E94DE1F82E060E040E020E00E94DE1F73
:104D400010921D0435992EC00E94752B882329F0DE
:104D5000809125048F5F80932504809125048436FB
:104D600008F41DC24298863908F419C20E94B92974
:104D7000882321F482E49EE00E943B2C10922504BB
:104D800080911B0490911C048F7B806290931C0483
:104D900080931B0480E061E040E020E00E94DE1F81
:104DA0008BE0FBC110922504429AF9C180910E0953
:104DB000882309F4F4C185E69EE00E943B2CC09054
:104DC0000B04D0900C04E0900D04F0900E040E94AF
:104DD00040248093260480910B0490910C048C193C
:104DE0009D090E946B2C80E89EE00E943B2C8091E4
:104DF00026040E9408230E94642A85E00E9429203C
:104E000081E080931E0480931504C9C1813009F4A8
:104E100044C084E89EE00E943B2C8091DF038B30ED
:104E200069F580912604882399F481E99EE00E9427
:104E30003B2C87E00E94292080911B0490911C0448
:104E4000806890931C0480931B0481E060E012C092
:104E500087EA9EE00E943B2C88E00E9429208091F6
:104E60001B0490911C04916090931C0480931B047C
:104E700081E061E040E020E00E94DE1F86EC9EE0E1
:104E80000E943B2C80911C040E94B42C80911B0436
:104E90000E94B42C81ED9EE07FC080911B0487FFAF
:104EA00035C080910E09882389F180911D048823E3
:104EB00061F00E947320882341F083ED9EE00E9400
:104EC0003B2C80E00E94292015C080911D0488237E
:104ED000A1F080911504882381F08091660980FDFE
:104EE0000CC08DEE9EE00E943B2C80E00E942920A9
:104EF0001092150482E080931E0480911A04882386
:104F000029F084E080931E0410921A04359B47C157
:104F10008BE09FE039C18230A1F080E29FE00E94E7
:104F20003B2C8DE29FE00E943B2C80911C040E9450
:104F3000B42C80911B040E94B42C8AE793E00E9459
:104F4000292C0E948520882351F088E39FE00E944D
:104F50003B2C81E00E94292081E080931E04359B38
:104F600009C08CE49FE00E943B2C86E00E9429202F
:104F700010921E0480911A04882309F410C184E061
:104F800080931E0410921A040AC18091DF038330BB
:104F900009F405C181E69FE00E943B2C00C180918D
:104FA000DF03843071F180911B0490911C048B7F8E
:104FB00090931C0480931B048EE69FE00E943B2C80
:104FC0008BE79FE00E943B2C80911C040E94B42C34
:104FD00080911B040E94B42C8AE793E00E94292C44
:104FE000469A1092250480911304882351F08CE096
:104FF00061E04CED53E00E94F42586E89FE00E94BA
:105000003B2C0E94752B882339F0809125048F3129
:1050100018F48F5F80932504809125048E3159F414
:105020008CE760E040E40E94932182E061E040E090
:1050300020E00E94DE1F0E9485208823A1F080913D
:105040001B0490911C0482608E7F90931C048093BB
:105050001B0481EA9FE00E943B2C81E00E942920F2
:1050600085E080931E0480911804882319F085E060
:1050700080931E04359B93C085EB9FE00E943B2CE0
:1050800086E00E94292080911304882309F481C0BE
:105090008CE061E048ED53E00E94F4258AEC9FE04B
:1050A0000E943B2C76C08091DF03853041F180EE79
:1050B0009FE00E943B2C8DEE9FE00E943B2C809154
:1050C0001C040E94B42C80911B040E94B42C8AE71B
:1050D00093E00E94292C82E060E040E020E00E9402
:1050E000DE1F80911304882351F08CE061E048EDCD
:1050F00053E00E94F42588EF9FE00E943B2C8091B2
:105100001804882389F080911B0490911C0484600A
:1051100090931C0480931B0487B18F7687B982E03B
:105120000E9429201092180480911904882329F0E4
:1051300086E080931E0410921904359B30C08EE0E7
:1051400090E122C08091DF038630D1F08CE760E4EB
:1051500040E40E949321469883E290E10E943B2C18
:1051600080E390E10E943B2C80911C040E94B42CAF
:1051700080911B040E94B42C8AE793E00E94292CA2
:10518000359B0AC08BE390E10E943B2C86E00E9495
:10519000292010921E0403C081E080931E04809198
:1051A0001604882309F443C080911B0480FF03C0C8
:1051B00080E00E94292080911B0481FF03C081E0D0
:1051C0000E94292080911B0482FF03C082E00E947C
:1051D000292080911B0483FF03C083E00E942920C3
:1051E00080911B0484FF03C084E00E9429208091E9
:1051F0001B0485FF03C085E00E94292080911B04C9
:1052000086FF03C086E00E94292080911B0487FF4F
:1052100003C087E00E94292080911B0490911C0408
:1052200090FF03C088E00E94292010921604FF908E
:10523000EF90DF90CF900895EF92FF921F93CF935E
:10524000DF930F92CDB7DEB7182F7A0169830E94E2
:10525000CF29812F880F0E94F22969818823E9F0E4
:10526000862F83700E94F2298823B9F00E94DA29E0
:10527000812F880F81600E94F229882371F081E0DC
:105280000E94282AF701808380E00E94282AF701E3
:1052900081830E94E72980E003C00E94E72981E022
:1052A0000F90DF91CF911F91FF90EF900895CF93D2
:1052B000DF9300D0CDB7DEB76A8389830E94CF2900
:1052C0008981880F0E94F2296A81882329F0862F1C
:1052D0000E94F229882321F40E94E72981E009C075
:1052E0000E94E7298FE097E20197F1F700C00000E4
:1052F00080E00F900F90DF91CF910895CF92DF92D1
:10530000EF92FF920F931F93CF93DF930F92CDB73E
:10531000DEB77B0189830E94CF298981880F816054
:105320000E94F229882321F40E94E7298FEF17C0F9
:1053300081E00E94282A182F00E080E00E94282A9D
:10534000C82EDD24C02AD12A0E94E729E114F104E5
:1053500011F48D2D04C0F701D182C08280E00F903E
:10536000DF91CF911F910F91FF90EF90DF90CF9041
:1053700008958BB18F7C8BB98AB18F7C8AB989E013
:1053800096E09A95F1F700C0549A96E09A95F1F755
:1053900000C054988150A1F789B180720895559A40
:1053A00086E08A95F1F700C0549A86E08A95F1F775
:1053B00000C00895559886E08A95F1F700C054988A
:1053C00086E08A95F1F700C00E94CF29089554988D
:1053D00086E08A95F1F700C0559886E08A95F1F746
:1053E00000C00895F89428E030E090E8492F482361
:1053F00011F4559A01C0559846E04A95F1F700C05E
:1054000054984DE04A95F1F70000549A46E04A95C9
:10541000F1F700C096952150304041F7559886E04D
:105420008A95F1F700C0549846E04A95F1F700C01C
:1054300099B186E08A95F1F700C0549A559A46E0F2
:105440004A95F1F700C0789481E095FD80E00895D9
:10545000282FF894559898E080E0880F36E03A9528
:10546000F1F700C0549836E03A95F1F700C04D9935
:10547000816036E03A95F1F700C0549A36E03A95EB
:10548000F1F700C0915049F7222311F0559A01C05D
:10549000559896E09A95F1F700C054983DE03A95FA
:1054A000F1F70000549A559A96E09A95F1F700C0EA
:1054B0007894089580912904882319F08BE090E076
:1054C000089589E090E0089581E08093290408958B
:1054D0001092290408958BB18F738BB98AB18F73A1
:1054E0008AB90895579A86E08A95F1F700C0569ACE
:1054F00086E08A95F1F700C00895579886E08A956E
:10550000F1F700C0569886E08A95F1F700C00E9436
:10551000722A0895569886E08A95F1F700C0579848
:1055200086E08A95F1F700C0089528E030E090E821
:10553000492F482311F4579A01C0579846E04A95DD
:10554000F1F700C056984DE04A95F1F70000569AE1
:1055500046E04A95F1F700C096952150304041F75A
:10556000579886E08A95F1F700C0569896E09A958C
:10557000F1F700C089B146E04A95F1F700C0569AAC
:10558000579A96E09A95F1F700C08095881F882772
:10559000881F0895282F579898E080E0880F36E0FC
:1055A0003A95F1F700C0569836E03A95F1F700C009
:1055B0004F99816036E03A95F1F700C0569A36E08F
:1055C0003A95F1F700C0915049F7222311F0579A0C
:1055D00001C0579896E09A95F1F700C056983DE0C3
:1055E0003A95F1F70000569A579A96E09A95F1F796
:1055F00000C008959091840983B180958927909186
:105600002A049823909590932A0420912B04282310
:10561000292720932B04982392238091840989279A
:105620008093840920918309809184098923822BA6
:105630008093830920918209809184098095892330
:10564000822B809382090895F8949091830989238D
:105650009091830998279093830978940895F894FA
:1056600090918209892390918209982790938209C9
:1056700078940895F89490918409789489230895F2
:105680008093300481E080932F04089510922F04BA
:10569000089581E090912F04992309F480E0089502
:1056A00080913004882329F081508093300480E079
:1056B000089581E0089580932E0481E080932D0465
:1056C000089510922D04089581E090912D0499235E
:1056D00009F480E0089581E090912E04911180E01A
:1056E000089581E080932C04089580912C048823F0
:1056F00021F010922C0481E0089580E0089510922A
:10570000C5008CE08093C40088E98093C1001092AA
:10571000070A1092050A1092060A1092880A089544
:105720009091050A2091070A91509F772917C1F39C
:10573000E091070AF0E0E85FF54F80838091070A67
:105740008F5F8093070A8091070A803811F41092C6
:10575000070A8091C10080628093C1000895309152
:10576000060A2091880A3217A1F02091880AE22FB8
:10577000F0E0EB57F64F3081FC0130832F5F209330
:10578000880A8091880A803831F41092880A80E073
:10579000089581E0089580E008951F920F920FB65A
:1057A0000F920BB60F9211248F939F93EF93FF9359
:1057B000E091050AF0E0E85FF54F80818093C60034
:1057C0008091050A8F5F8093050A8091050A8038D1
:1057D00011F41092050A9091070A8091050A981712
:1057E00029F48091C1008F7D8093C100FF91EF91DA
:1057F0009F918F910F900BBE0F900FBE0F901F9037
:1058000018951F920F920FB60F920BB60F9211249C
:105810008F939F93EF93FF938091060AE82FF0E018
:105820009091C600EB57F64F90838F5F8093060AE6
:105830008091060A803811F41092060AFF91EF91C8
:105840009F918F910F900BBE0F900FBE0F901F90E6
:105850001895CF93DF93EC0108C08A3019F48DE0DE
:105860000E94902B89910E94902B88818823A9F710
:10587000DF91CF9108951F93CF93DF93EC01219691
:10588000FC0114911A3019F48DE00E94902B812FA5
:105890000E94902BFE0121961491112399F7DF911C
:1058A000CF911F9108950F931F93CF93DF93082FEC
:1058B000C8E0D0E010E8812F802311F081E301C01F
:1058C00080E30E94902B16952197A9F7DF91CF9145
:1058D0001F910F910895DF92EF92FF920F931F9304
:1058E000CF93DF93CDB7DEB729970FB6F894DEBF1D
:1058F0000FBECDBF8C01DE011196E1EEF3E088E032
:1059000001900D928150E1F77E010894E11CF11C99
:1059100084E0D82E91E010C08F5F021B130B90E043
:1059200002171307C8F7992329F4805D99870E940D
:10593000902B9985DA9431F0F701219131917F0113
:1059400080E0EECF802F805D0E94902B29960FB6CD
:10595000F894DEBF0FBECDBFDF91CF911F910F91A5
:10596000FF90EF90DF9008951F93CF93DF93CDB713
:10597000DEB760970FB6F894DEBF0FBECDBF182F0D
:10598000DE011196E9EEF3E080E101900D92815085
:10599000E1F7812F82958F70E1E0F0E0EC0FFD1FC1
:1059A000E80FF11D80810E94902B1F70E1E0F0E074
:1059B000EC0FFD1FE10FF11D80810E94902B60967E
:1059C0000FB6F894DEBF0FBECDBFDF91CF911F9110
:1059D0000895CF93DF93CDB7DEB7C354D0400FB651
:1059E000F894DEBF0FBECDBF10920E0980E880BFD5
:1059F000A89528E288E190E00FB6F894A8958093E6
:105A000060000FBE209360001092120910921309DB
:105A10001092140910921509109218090E947F2BF8
:105A20000E9476080E946B2A0E94D61F90931D093F
:105A300080931C0989E0809381008FE39FE190931C
:105A400089008093880082E080936F002C9885B154
:105A5000806685B984B1806784B94098389A139A72
:105A6000149881B1886181B915980D9A46983E9A2B
:105A70005A9852985B98539A429A3A9A88B18F767C
:105A800088B987B18F7687B980E060E14AE454E055
:105A900022E534E00E94011181E060E24AE354E033
:105AA00022E634E00E94011182E060E442E454E026
:105AB0002AE534E00E94011110921609789481EED3
:105AC00093E00E943B2C109211098DE193E00E941B
:105AD000292C0E94B60E0E946B2C8AEF93E00E9444
:105AE0003B2C8CEF93E00E943B2C809160000E9445
:105AF000B42C85E094E00E943B2C87E094E00E9467
:105B00003B2C84E393E00E94292C80E194E00E94E6
:105B10003B2C86E294E00E943B2C8CE294E00E94B5
:105B20003B2C8CE394E00E943B2C82E494E00E94A6
:105B30003B2C8DE494E00E943B2C86E594E00E948F
:105B40003B2C8BE594E00E943B2C87E694E00E947E
:105B50003B2C8BE694E00E943B2C84E794E00E946F
:105B60003B2C86E794E00E943B2C84B70E94B42C27
:105B70008EE794E00E943B2C14BE0E94D3138093C6
:105B800017090E94590F8AE393E00E94292C809103
:105B900017090E94B42C8BE493E00E94292C0E94E8
:105BA000210E80E2809362091092630900E010E008
:105BB000FF24FA94A8950E945A0E0E943E098091F3
:105BC0000C098823B1F080E969E079E00E942E1386
:105BD00082E96FE079E00E942E130E945A2A8A30EF
:105BE000910528F088E46AE179E00E947E2910920C
:105BF0000C090E942D2680910D09882321F00E9416
:105C0000E32010920D090E94690F882311F0A895D6
:105C1000FACF0E94D90F80911C0990911D09FC01B7
:105C2000208120FF2AC00E944814E0911C09F091B5
:105C30001D0990819E7F90838823F9F4CF010E94F3
:105C4000151420911C0930911D09882389F4C9017C
:105C5000BE016F5F7F4F0E946F14882371F0CE01E9
:105C600001960E941B14CE0101960E94DD1005C012
:105C7000C9010E94D91F0E94FB1080911909882335
:105C800009F498CF0E94492B882379F00E94502B69
:105C9000882359F081E0809316090E94462B80E802
:105CA00094E00E943B2C00E010E08091120990915A
:105CB0001309A0911409B09115090196A11DB11DF8
:105CC0008093120990931309A0931409B0931509B6
:105CD00080E00E94B81181E00E94B81182E00E9429
:105CE000B81180911609843009F454C0853040F40D
:105CF0008130B9F0813070F0833009F08EC031C04E
:105D0000863009F47CC0863008F461C0873009F021
:105D100084C077C00D9A389A139A14981092180973
:105D20007CC080E00E94EA08F2E08C3B9F0708F408
:105D300074C00F5F1F4F0230110509F06EC083E081
:105D4000809316091398149A8AE994E00E943B2CD8
:105D500080911209909113090E946B2C83EC94E0BE
:105D600016C00F5F1F4F0531110508F456C0389853
:105D700084E08093160986EC94E00E943B2C80918D
:105D80001209909113090E946B2C86EF94E00E94F7
:105D90003B2C41C0319B41C081E080930E090F5FD5
:105DA0001F4F06301105C8F10D9885E08093160944
:105DB00089EF94E00E943B2C809112099091130985
:105DC0000E946B2C87E295E00E943B2C26C08091BC
:105DD0001809882311F58AE295E00E943B2C8091F6
:105DE0001209909113090E946B2C8DE395E00E949B
:105DF0003B2C0E94EC0E81E0809318090EC00D9A96
:105E00000CC0389A139A149881E08093110910926B
:105E100016091092180900E010E0E0901609FE142F
:105E200009F441C022E0E216B9F02E1530F081E00D
:105E3000EE2071F0E816B9F50AC0E5E0EE16E1F0E3
:105E4000F7E0EF1621F124E0E21669F50AC081E0DF
:105E500060E041E050E01FC081E060E042E050E0DF
:105E60001AC081E060E040E050E00E941B1182E037
:105E700060E042E050E015C081E060E040E050E0CA
:105E80000E941B1182E060E041E050E00AC081E026
:105E900060E040E050E00E941B1182E060E040E0E2
:105EA00050E00E941B1110921909FE2C83CE629FB4
:105EB000D001739FF001829FE00DF11D649FE00D02
:105EC000F11D929FF00D839FF00D749FF00D659F63
:105ED000F00D9927729FB00DE11DF91F639FB00D62
:105EE000E11DF91FBD01CF0111240895991B79E02F
:105EF00004C0991F961708F0961B881F7A95C9F75A
:105F00008095089597FB092E07260AD077FD04D0C7
:105F10000CD006D000201AF4709561957F4F08953B
:105F2000F6F7909581959F4F0895AA1BBB1B51E1F1
:105F300007C0AA1FBB1FA617B70710F0A61BB70BF9
:105F4000881F991F5A95A9F780959095BC01CD019E
:105F50000895FB01DC0102C005900D9241505040B4
:105F6000D8F70895FB01DC0104C08D9101908019E0
:105F700021F441505040C8F7881B990B0895FB014C
:105F8000DC0102C001900D9241505040D8F70895B5
:105F9000DC01CB01FC01F999FECF06C0F2BDE1BDE9
:105FA000F89A319600B40D9241505040B8F70895D8
:105FB000F999FECF92BD81BDF89A992780B50895D1
:105FC000DC01CB0103C02D910E94EB2F41505040CA
:105FD000D0F70895262FF999FECF1FBA92BD81BD43
:105FE00020BD0FB6F894FA9AF99A0FBE019608955B
:045FF000F894FFCF53
:105FF4000A0001FFFF204552524F5221003A20303F
:1060040078000A002E2E2E204552524F52210A00AB
:106014002E2E2E20646F6E65210A00646F6E65213A
:106024000A00205265616420556E697175652D49B9
:10603400443A200020525F4552524F522100206DB5
:10604400560A0020000A0A383330304C3E0A0075E4
:106054006E6B6E6F776E20636F6D6D616E640A0098
:10606400383330304C3E00535441540048454C5072
:106074000052544D310052544D320052544D3300AD
:1060840052544D340052544D350052544D36005242
:10609400544D370052544D3800564F4C5400505212
:1060A4004F4D00494400444143570044414352008A
:1060B400007702D50D7C02E90B8102AE0D860287C2
:1060C4000D8B02750D90026C0D9502630D9A025AA8
:1060D4000D9F02E30BA4021B0DA902C50CAE0269BD
:1060E4000CB302830CB6021A0CBB02EF0BC0020005
:1060F400000A00726571206F75742064726F70708D
:10610400656420616674657220330A000A4D6F6409
:10611400756C652053657269616C204E756D62659E
:10612400723A2000322E372E35004D6F64756C653F
:1061340020416464726573733A20000A0A000A00FD
:106144006F6666733A0020636E743A002000322E44
:10615400372E350036061B068E07DB054E070E0765
:10616400CE069B055B058E064E060A0072746D20F2
:10617400636D6E206864722063686B206661696C6D
:106184000A006D756C7420686561646572206368CB
:1061940065636B73756D206572726F72210A0020DE
:1061A400004452544D2D44574338004452544D2D0D
:1061B4004453380052544D2D44574300B10309034E
:1061C400BB030803C403070320002FFC2C1C06FF99
:1061D400FF1027E80364000A0030313233343536C7
:0A61E4003738394142434445460074
:00000001FF
